BL51 BANKED LINKER/LOCATER V5.00                                                        02/17/2010  13:07:02  PAGE 1


BL51 BANKED LINKER/LOCATER V5.00, INVOKED BY:
C:\KEIL\C51\BIN\BL51.EXE Automat.obj TO Aparat za slatkise


MEMORY MODEL: SMALL


INPUT MODULES INCLUDED:
  Automat.obj (AUTOMAT)
  C:\KEIL\C51\LIB\C51S.LIB (?C_STARTUP)
  C:\KEIL\C51\LIB\C51S.LIB (?C?COPY)
  C:\KEIL\C51\LIB\C51S.LIB (?C?SCDIV)
  C:\KEIL\C51\LIB\C51S.LIB (?C?CLDOPTR)
  C:\KEIL\C51\LIB\C51S.LIB (?C?IMUL)
  C:\KEIL\C51\LIB\C51S.LIB (?C?SIDIV)
  C:\KEIL\C51\LIB\C51S.LIB (?C?IILDX)
  C:\KEIL\C51\LIB\C51S.LIB (?C_XBP)
  C:\KEIL\C51\LIB\C51S.LIB (?C?ADDXBP)
  C:\KEIL\C51\LIB\C51S.LIB (STRCAT)
  C:\KEIL\C51\LIB\C51S.LIB (?C_INIT)
  C:\KEIL\C51\LIB\C51S.LIB (?C?CLDPTR)
  C:\KEIL\C51\LIB\C51S.LIB (?C?CSTPTR)
  C:\KEIL\C51\LIB\C51S.LIB (?C?UIDIV)


LINK MAP OF MODULE:  Aparat za slatkise (AUTOMAT)


            TYPE    BASE      LENGTH    RELOCATION   SEGMENT NAME
            -----------------------------------------------------

            * * * * * * *   D A T A   M E M O R Y   * * * * * * *
            REG     0000H     0008H     ABSOLUTE     "REG BANK 0"
            DATA    0008H     000FH     UNIT         _DATA_GROUP_
            DATA    0017H     0002H     UNIT         ?C?LIB_DATA
                    0019H     0007H                  *** GAP ***
            BIT     0020H.0   0001H.3   UNIT         ?BI?AUTOMAT
                    0021H.3   0000H.5                *** GAP ***
            DATA    0022H     0031H     UNIT         ?DT?AUTOMAT
            IDATA   0053H     0001H     UNIT         ?STACK

            * * * * * * *  X D A T A   M E M O R Y  * * * * * * *
            XDATA   0000H     0773H     UNIT         ?XD?AUTOMAT
            XDATA   0773H     0003H     UNIT         _XDATA_GROUP_

            * * * * * * *   C O D E   M E M O R Y   * * * * * * *
            CODE    0000H     0003H     ABSOLUTE     
            CODE    0003H     0003H     ABSOLUTE     
                    0006H     0005H                  *** GAP ***
            CODE    000BH     0003H     ABSOLUTE     
                    000EH     0005H                  *** GAP ***
            CODE    0013H     0003H     ABSOLUTE     
                    0016H     0005H                  *** GAP ***
            CODE    001BH     0003H     ABSOLUTE     
                    001EH     0005H                  *** GAP ***
            CODE    0023H     0003H     ABSOLUTE     
                    0026H     07DAH                  *** GAP ***
            CODE    0800H     0247H     UNIT         ?C?LIB_CODE
BL51 BANKED LINKER/LOCATER V5.00                                                      02/17/2010  13:07:02  PAGE 2


            CODE    0A47H     0232H     UNIT         ?PR?SERIJSKI_PORT?AUTOMAT
            CODE    0C79H     01A9H     UNIT         ?PR?_?EXTERN0_TASTATURA?AUTOMAT
            CODE    0E22H     00C8H     UNIT         ?PR?FORMIRAJ_ISPIS?AUTOMAT
            CODE    0EEAH     00C0H     UNIT         ?CO?AUTOMAT
            CODE    0FAAH     00BCH     UNIT         ?PR?TIMER0_1MS_PREKID?AUTOMAT
            CODE    1066H     00B9H     UNIT         ?PR?VRATI_KUSUR?AUTOMAT
            CODE    111FH     00B6H     UNIT         ?PR?_ISPISI_PORUKU_NA_DISPLEJU?AUTOMAT
            CODE    11D5H     0093H     UNIT         ?PR?PROCITAJ_VREDNOST_IZ_AUTOMATA?AUTOMAT
            CODE    1268H     008CH     UNIT         ?C_C51STARTUP
            CODE    12F4H     0086H     UNIT         ?PR?FORMIRAJ_VREME?AUTOMAT
            CODE    137AH     007BH     UNIT         ?PR?PRIKAZI_PORUKU_O_PROIZVODU?AUTOMAT
            CODE    13F5H     0058H     UNIT         ?PR?_STRCAT?STRCAT
            CODE    144DH     0038H     UNIT         ?PR?MAIN?AUTOMAT
            CODE    1485H     0027H     UNIT         ?PR?UCITAJ_TASTER?AUTOMAT
            CODE    14ACH     0023H     UNIT         ?PR?EXTERN1_AUTOMAT_SPIRALA?AUTOMAT
            CODE    14CFH     0014H     UNIT         ?PR?CEKAJ_1MSEC?AUTOMAT
            CODE    14E3H     0011H     UNIT         ?PR?_IZBACI_NOVCANICU?AUTOMAT
            CODE    14F4H     0011H     UNIT         ?C_INITSEG
            CODE    1505H     0010H     UNIT         ?PR?NA_POCETNO_STANJE?AUTOMAT
            CODE    1515H     000CH     UNIT         ?PR?TIMER1_1MS_POSLE_STARTOVANJA?AUTOMAT
            CODE    1521H     0009H     UNIT         ?PR?POKRENI_TIMER?AUTOMAT



OVERLAY MAP OF MODULE:   Aparat za slatkise (AUTOMAT)


SEGMENT                                            DATA_GROUP          XDATA_GROUP
  +--> CALLED SEGMENT                            START    LENGTH     START    LENGTH
------------------------------------------------------------------------------------
?PR?TIMER0_1MS_PREKID?AUTOMAT                    -----    -----      -----    -----
  +--> ?PR?FORMIRAJ_VREME?AUTOMAT
  +--> ?PR?POKRENI_TIMER?AUTOMAT

?PR?FORMIRAJ_VREME?AUTOMAT                       -----    -----      -----    -----
  +--> ?CO?AUTOMAT

*** NEW ROOT ***************************************************

?PR?EXTERN1_AUTOMAT_SPIRALA?AUTOMAT              -----    -----      -----    -----
  +--> ?PR?PROCITAJ_VREDNOST_IZ_AUTOMATA?AUT...

?PR?PROCITAJ_VREDNOST_IZ_AUTOMATA?AUT...         -----    -----      -----    -----
  +--> ?PR?_IZBACI_NOVCANICU?AUTOMAT
  +--> ?PR?CEKAJ_1MSEC?AUTOMAT

?PR?_IZBACI_NOVCANICU?AUTOMAT                    -----    -----      -----    -----
  +--> ?PR?CEKAJ_1MSEC?AUTOMAT

?PR?CEKAJ_1MSEC?AUTOMAT                          -----    -----      -----    -----
  +--> ?PR?POKRENI_TIMER?AUTOMAT

*** NEW ROOT ***************************************************

?PR?_?EXTERN0_TASTATURA?AUTOMAT                  -----    -----      -----    -----
  +--> ?PR?UCITAJ_TASTER?AUTOMAT
  +--> ?CO?AUTOMAT
BL51 BANKED LINKER/LOCATER V5.00                                                      02/17/2010  13:07:02  PAGE 3


  +--> ?PR?_ISPISI_PORUKU_NA_DISPLEJU?AUTOMAT
  +--> ?PR?VRATI_KUSUR?AUTOMAT
  +--> ?PR?NA_POCETNO_STANJE?AUTOMAT
  +--> ?PR?FORMIRAJ_ISPIS?AUTOMAT
  +--> ?PR?PRIKAZI_PORUKU_O_PROIZVODU?AUTOMAT

?PR?UCITAJ_TASTER?AUTOMAT                        -----    -----      -----    -----
  +--> ?CO?AUTOMAT

?PR?_ISPISI_PORUKU_NA_DISPLEJU?AUTOMAT           0008H    000FH      -----    -----
  +--> ?CO?AUTOMAT

?PR?VRATI_KUSUR?AUTOMAT                          -----    -----      -----    -----
  +--> ?PR?PROCITAJ_VREDNOST_IZ_AUTOMATA?AUT...
  +--> ?CO?AUTOMAT
  +--> ?PR?_ISPISI_PORUKU_NA_DISPLEJU?AUTOMAT

?PR?PRIKAZI_PORUKU_O_PROIZVODU?AUTOMAT           -----    -----      -----    -----
  +--> ?CO?AUTOMAT
  +--> ?PR?_STRCAT?STRCAT
  +--> ?PR?_ISPISI_PORUKU_NA_DISPLEJU?AUTOMAT

?PR?_STRCAT?STRCAT                               0008H    0009H      -----    -----

*** NEW ROOT ***************************************************

?PR?SERIJSKI_PORT?AUTOMAT                        -----    -----      0773H    0003H

*** NEW ROOT ***************************************************

?C_C51STARTUP                                    -----    -----      -----    -----
  +--> ?PR?MAIN?AUTOMAT
  +--> ?C_INITSEG



SYMBOL TABLE OF MODULE:  Aparat za slatkise (AUTOMAT)

  VALUE           TYPE          NAME
  ----------------------------------

  -------         MODULE        AUTOMAT
  C:0000H         SYMBOL        _ICE_DUMMY_
  D:0080H         PUBLIC        P0
  C:0F95H         PUBLIC        tasteri
  D:0090H         PUBLIC        P1
  C:1521H         PUBLIC        pokreni_timer
  B:0090H.1       PUBLIC        LE_START
  D:00A0H         PUBLIC        P2
  C:14E3H         PUBLIC        _izbaci_novcanicu
  B:00B0H.4       PUBLIC        T0
  B:00D0H.6       PUBLIC        AC
  B:00B0H.5       PUBLIC        T1
  B:0090H.3       PUBLIC        SEL_moneyD0_KD0
  B:00A8H.7       PUBLIC        EA
  D:0022H         PUBLIC        trenutno_vreme
  D:002AH         PUBLIC        trenutni_ispis
BL51 BANKED LINKER/LOCATER V5.00                                                      02/17/2010  13:07:02  PAGE 4


  D:00A8H         PUBLIC        IE
  D:0032H         PUBLIC        kodovi
  D:003AH         PUBLIC        prikazuj_vreme_ispis_poruku
  C:0A47H         PUBLIC        serijski_port
  B:0020H.0       PUBLIC        pokrenut_motor
  B:00B0H.7       PUBLIC        RD
  C:1505H         PUBLIC        na_pocetno_stanje
  D:003BH         PUBLIC        taster
  B:00A8H.4       PUBLIC        ES
  B:0098H.0       PUBLIC        RI
  B:00B0H.2       PUBLIC        INT0
  B:00D0H.7       PUBLIC        CY
  B:0098H.1       PUBLIC        TI
  B:00B0H.3       PUBLIC        INT1
  B:0020H.1       PUBLIC        nema_novcanice10
  B:0020H.2       PUBLIC        nema_novcanice20
  B:00B8H.4       PUBLIC        PS
  B:00D0H.2       PUBLIC        OV
  B:0020H.3       PUBLIC        nema_novcanice50
  C:144DH         PUBLIC        main
  B:00B0H.6       PUBLIC        WR
  C:0C79H         PUBLIC        _?extern0_tastatura
  D:003CH         PUBLIC        broj_poruke
  X:0000H         PUBLIC        msec
  C:0FAAH         PUBLIC        timer0_1ms_prekid
  D:0099H         PUBLIC        SBUF
  D:0087H         PUBLIC        PCON
  C:137AH         PUBLIC        prikazi_poruku_o_proizvodu
  X:0002H         PUBLIC        sati
  D:0098H         PUBLIC        SCON
  D:0089H         PUBLIC        TMOD
  D:0088H         PUBLIC        TCON
  D:003DH         PUBLIC        suma
  D:003FH         PUBLIC        novcanica
  D:0040H         PUBLIC        cifra1
  D:0041H         PUBLIC        trenutni_karakter
  D:0042H         PUBLIC        cifra2
  C:0F8DH         PUBLIC        nepodeseno_vreme
  B:0020H.4       PUBLIC        nema_novcanica
  X:0003H         PUBLIC        sec
  C:14CFH         PUBLIC        cekaj_1msec
  B:0088H.1       PUBLIC        IE0
  B:0088H.3       PUBLIC        IE1
  X:0004H         PUBLIC        zarade_proizvoda
  B:0090H.4       PUBLIC        moneyD0_KD0
  B:0090H.7       PUBLIC        KD3
  B:0090H.5       PUBLIC        moneyD1_KD1
  C:0FA2H         SYMBOL        _?ix1000
  C:11DDH         PUBLIC        procitaj_vrednost_iz_automata
  B:0090H.6       PUBLIC        moneyD2_KD2
  X:00CCH         PUBLIC        min
  C:1066H         PUBLIC        vrati_kusur
  B:00A8H.1       PUBLIC        ET0
  B:00A8H.3       PUBLIC        ET1
  B:0088H.5       PUBLIC        TF0
  X:00CDH         PUBLIC        ukupno_zaradjeno
  B:0088H.7       PUBLIC        TF1
BL51 BANKED LINKER/LOCATER V5.00                                                      02/17/2010  13:07:02  PAGE 5


  B:0098H.2       PUBLIC        RB8
  D:008CH         PUBLIC        TH0
  B:00A8H.0       PUBLIC        EX0
  B:0088H.0       PUBLIC        IT0
  D:008DH         PUBLIC        TH1
  B:0098H.3       PUBLIC        TB8
  B:00A8H.2       PUBLIC        EX1
  B:0088H.2       PUBLIC        IT1
  B:00D0H.0       PUBLIC        P
  B:0098H.7       PUBLIC        SM0
  D:008AH         PUBLIC        TL0
  B:0098H.6       PUBLIC        SM1
  D:008BH         PUBLIC        TL1
  B:0020H.5       PUBLIC        nema_novcanice100
  B:0098H.5       PUBLIC        SM2
  B:0020H.6       PUBLIC        nema_novcanice200
  B:00B8H.1       PUBLIC        PT0
  B:0090H.2       PUBLIC        LE_MONEY_OUT
  B:00B8H.3       PUBLIC        PT1
  B:00D0H.3       PUBLIC        RS0
  B:0088H.4       PUBLIC        TR0
  B:00D0H.4       PUBLIC        RS1
  B:0088H.6       PUBLIC        TR1
  B:00B8H.0       PUBLIC        PX0
  B:00B8H.2       PUBLIC        PX1
  X:00CFH         PUBLIC        nazivi_proizvoda
  B:0020H.7       PUBLIC        novcanica_izbacena
  B:0021H.0       PUBLIC        kupljen_proizvod
  C:12F4H         PUBLIC        formiraj_vreme
  X:070FH         PUBLIC        cene_proizvoda
  D:0043H         PUBLIC        Hpromet
  B:0021H.1       PUBLIC        oneMS
  C:1515H         PUBLIC        timer1_1ms_posle_startovanja
  B:0021H.2       PUBLIC        vreme_podeseno
  B:0098H.4       PUBLIC        REN
  D:0044H         PUBLIC        Lpromet
  D:0045H         PUBLIC        trenutni_simbol
  C:0E22H         PUBLIC        formiraj_ispis
  D:0046H         PUBLIC        trenutna_poruka
  D:004EH         PUBLIC        trenutno_stanje
  D:004FH         PUBLIC        MASKA
  B:00B0H.0       PUBLIC        RXD
  B:0090H.0       PUBLIC        LE_DISPL
  B:00B0H.1       PUBLIC        TXD
  D:0050H         PUBLIC        broj_proizvoda
  D:0051H         PUBLIC        brojac
  B:00D0H.5       PUBLIC        F0
  C:111FH         PUBLIC        _ispisi_poruku_na_displeju
  D:0052H         PUBLIC        uneto_cifara
  C:1485H         PUBLIC        ucitaj_taster
  C:14ACH         PUBLIC        extern1_automat_spirala
  -------         PROC          MAIN
  C:144DH         LINE#         105
  C:144DH         LINE#         107
  C:144FH         LINE#         108
  C:1456H         LINE#         109
  C:1458H         LINE#         110
BL51 BANKED LINKER/LOCATER V5.00                                                      02/17/2010  13:07:02  PAGE 6


  C:145AH         LINE#         111
  C:145DH         LINE#         113
  C:145FH         LINE#         114
  C:1461H         LINE#         116
  C:1463H         LINE#         117
  C:1465H         LINE#         119
  C:1467H         LINE#         120
  C:1469H         LINE#         122
  C:146CH         LINE#         123
  C:146FH         LINE#         125
  C:1472H         LINE#         126
  C:1475H         LINE#         128
  C:1478H         LINE#         129
  C:147BH         LINE#         131
  C:147EH         LINE#         132
  C:1480H         LINE#         134
  C:1483H         LINE#         136
  -------         ENDPROC       MAIN
  -------         PROC          POKRENI_TIMER
  C:1521H         LINE#         139
  C:1521H         LINE#         140
  C:1524H         LINE#         141
  C:1527H         LINE#         142
  C:1529H         LINE#         143
  -------         ENDPROC       POKRENI_TIMER
  -------         PROC          CEKAJ_1MSEC
  C:14CFH         LINE#         145
  C:14CFH         LINE#         146
  C:14D2H         LINE#         148
  C:14D5H         LINE#         149
  C:14D8H         LINE#         150
  C:14DBH         LINE#         151
  C:14DDH         LINE#         152
  C:14DFH         LINE#         154
  C:14E2H         LINE#         155
  -------         ENDPROC       CEKAJ_1MSEC
  -------         PROC          UCITAJ_TASTER
  C:1485H         LINE#         158
  C:1485H         LINE#         159
  C:1487H         LINE#         160
  C:148DH         LINE#         161
  C:14A0H         LINE#         163
  C:14A8H         LINE#         164
  C:14ABH         LINE#         165
  -------         ENDPROC       UCITAJ_TASTER
  -------         PROC          FORMIRAJ_ISPIS
  C:0E22H         LINE#         167
  C:0E22H         LINE#         168
  C:0E27H         LINE#         169
  C:0E2AH         LINE#         170
  C:0E2DH         LINE#         171
  C:0E2FH         LINE#         172
  C:0E34H         LINE#         173
  C:0E37H         LINE#         174
  C:0E37H         LINE#         175
  C:0E39H         LINE#         176
  C:0E39H         LINE#         177
BL51 BANKED LINKER/LOCATER V5.00                                                      02/17/2010  13:07:02  PAGE 7


  C:0E3CH         LINE#         178
  C:0E3FH         LINE#         179
  C:0E3FH         LINE#         181
  C:0E4CH         LINE#         182
  C:0E72H         LINE#         183
  C:0EA6H         LINE#         184
  C:0EDBH         LINE#         186
  C:0EDFH         LINE#         187
  C:0EE2H         LINE#         188
  C:0EE6H         LINE#         189
  C:0EE9H         LINE#         190
  C:0EE9H         LINE#         191
  C:0EE9H         LINE#         192
  -------         ENDPROC       FORMIRAJ_ISPIS
  -------         PROC          FORMIRAJ_VREME
  C:12F4H         LINE#         194
  C:12F4H         LINE#         195
  C:12F7H         LINE#         196
  C:1305H         LINE#         197
  C:1312H         LINE#         198
  C:1315H         LINE#         199
  C:1323H         LINE#         200
  C:1330H         LINE#         201
  C:1333H         LINE#         202
  C:1341H         LINE#         203
  C:134EH         LINE#         204
  C:134FH         LINE#         205
  C:134FH         LINE#         206
  C:1356H         LINE#         207
  C:135BH         LINE#         208
  C:1360H         LINE#         209
  C:1365H         LINE#         210
  C:136AH         LINE#         211
  C:136FH         LINE#         212
  C:1374H         LINE#         213
  C:1379H         LINE#         214
  C:1379H         LINE#         215
  -------         ENDPROC       FORMIRAJ_VREME
  -------         PROC          _IZBACI_NOVCANICU
  D:0007H         SYMBOL        novcanica
  -------         DO            
  D:0007H         SYMBOL        temp
  -------         ENDDO         
  C:14E3H         LINE#         217
  C:14E3H         LINE#         218
  C:14E8H         LINE#         219
  C:14ECH         LINE#         220
  C:14EEH         LINE#         221
  C:14F1H         LINE#         222
  C:14F3H         LINE#         223
  -------         ENDPROC       _IZBACI_NOVCANICU
  C:11D5H         SYMBOL        L?0161
  -------         PROC          L?0160
  -------         ENDPROC       L?0160
  C:11D5H         SYMBOL        L?0161
  -------         PROC          PROCITAJ_VREDNOST_IZ_AUTOMATA
  C:11DDH         LINE#         226
BL51 BANKED LINKER/LOCATER V5.00                                                      02/17/2010  13:07:02  PAGE 8


  C:11DDH         LINE#         227
  C:11E0H         LINE#         228
  C:11E2H         LINE#         229
  C:11E5H         LINE#         230
  C:11E7H         LINE#         231
  C:11E9H         LINE#         232
  C:11F9H         LINE#         233
  C:1209H         LINE#         234
  C:1219H         LINE#         235
  C:1229H         LINE#         236
  C:1242H         LINE#         238
  C:1252H         LINE#         239
  C:1260H         LINE#         241
  C:1263H         LINE#         242
  C:1265H         LINE#         243
  C:1267H         LINE#         244
  -------         ENDPROC       PROCITAJ_VREDNOST_IZ_AUTOMATA
  -------         PROC          _ISPISI_PORUKU_NA_DISPLEJU
  D:0008H         SYMBOL        poruka
  -------         DO            
  D:000BH         SYMBOL        temp
  D:0007H         SYMBOL        temp_sec
  D:000CH         SYMBOL        i
  D:000DH         SYMBOL        j
  D:000EH         SYMBOL        temp_poruka
  D:0016H         SYMBOL        len
  -------         ENDDO         
  C:111FH         LINE#         246
  C:1125H         LINE#         247
  C:1128H         LINE#         249
  C:112BH         LINE#         250
  C:112DH         LINE#         251
  C:113EH         LINE#         252
  C:1141H         LINE#         253
  C:1144H         LINE#         255
  C:1169H         LINE#         256
  C:116CH         LINE#         257
  C:116FH         LINE#         258
  C:1172H         LINE#         259
  C:1175H         LINE#         260
  C:1178H         LINE#         261
  C:117BH         LINE#         262
  C:117EH         LINE#         263
  C:1181H         LINE#         264
  C:118DH         LINE#         266
  C:1190H         LINE#         267
  C:119EH         LINE#         268
  C:11A5H         LINE#         269
  C:11CCH         LINE#         270
  C:11D1H         LINE#         272
  C:11D4H         LINE#         273
  -------         ENDPROC       _ISPISI_PORUKU_NA_DISPLEJU
  -------         PROC          VRATI_KUSUR
  C:1066H         LINE#         276
  C:1066H         LINE#         277
  C:1066H         LINE#         278
  C:1076H         LINE#         279
BL51 BANKED LINKER/LOCATER V5.00                                                      02/17/2010  13:07:02  PAGE 9


  C:1079H         LINE#         280
  C:1079H         LINE#         281
  C:1079H         LINE#         282
  C:107CH         LINE#         283
  C:1081H         LINE#         284
  C:1083H         LINE#         285
  C:1086H         LINE#         286
  C:1096H         LINE#         287
  C:1099H         LINE#         288
  C:1099H         LINE#         289
  C:1099H         LINE#         290
  C:109CH         LINE#         291
  C:10A1H         LINE#         292
  C:10A3H         LINE#         293
  C:10A6H         LINE#         294
  C:10B6H         LINE#         295
  C:10B9H         LINE#         296
  C:10B9H         LINE#         297
  C:10B9H         LINE#         298
  C:10BCH         LINE#         299
  C:10C1H         LINE#         300
  C:10C3H         LINE#         301
  C:10C5H         LINE#         302
  C:10D5H         LINE#         303
  C:10D8H         LINE#         304
  C:10D8H         LINE#         305
  C:10D8H         LINE#         306
  C:10DBH         LINE#         307
  C:10E0H         LINE#         308
  C:10E2H         LINE#         309
  C:10E4H         LINE#         310
  C:10F4H         LINE#         311
  C:10F7H         LINE#         312
  C:10F7H         LINE#         313
  C:10F7H         LINE#         314
  C:10FAH         LINE#         315
  C:10FDH         LINE#         316
  C:1103H         LINE#         317
  C:1105H         LINE#         318
  C:1105H         LINE#         319
  C:1105H         LINE#         320
  C:110BH         LINE#         321
  C:1114H         LINE#         322
  C:1114H         LINE#         323
  C:1114H         LINE#         324
  C:111EH         LINE#         325
  -------         ENDPROC       VRATI_KUSUR
  -------         PROC          PRIKAZI_PORUKU_O_PROIZVODU
  C:137AH         LINE#         327
  C:137AH         LINE#         328
  C:13EBH         LINE#         329
  C:13F4H         LINE#         331
  -------         ENDPROC       PRIKAZI_PORUKU_O_PROIZVODU
  -------         PROC          NA_POCETNO_STANJE
  C:1505H         LINE#         333
  C:1505H         LINE#         334
  C:1507H         LINE#         335
BL51 BANKED LINKER/LOCATER V5.00                                                      02/17/2010  13:07:02  PAGE 10


  C:150AH         LINE#         336
  C:150CH         LINE#         337
  C:150EH         LINE#         338
  C:1511H         LINE#         339
  C:1514H         LINE#         340
  -------         ENDPROC       NA_POCETNO_STANJE
  -------         PROC          TIMER0_1MS_PREKID
  C:0FAAH         LINE#         344
  C:0FC7H         LINE#         345
  C:0FCAH         LINE#         346
  C:0FCDH         LINE#         347
  C:0FE3H         LINE#         348
  C:0FE9H         LINE#         349
  C:0FEFH         LINE#         350
  C:0FF3H         LINE#         351
  C:0FF5H         LINE#         352
  C:0FFBH         LINE#         353
  C:0FFFH         LINE#         354
  C:1001H         LINE#         355
  C:1007H         LINE#         356
  C:100BH         LINE#         357
  C:100DH         LINE#         358
  C:100DH         LINE#         359
  C:100DH         LINE#         360
  C:100DH         LINE#         361
  C:100DH         LINE#         362
  C:1010H         LINE#         364
  C:101DH         LINE#         365
  C:1020H         LINE#         366
  C:1028H         LINE#         367
  C:1031H         LINE#         368
  C:1039H         LINE#         369
  C:1041H         LINE#         370
  C:1043H         LINE#         371
  C:1045H         LINE#         373
  C:1048H         LINE#         374
  C:104BH         LINE#         375
  -------         ENDPROC       TIMER0_1MS_PREKID
  -------         PROC          TIMER1_1MS_POSLE_STARTOVANJA
  C:1515H         LINE#         377
  C:1515H         LINE#         378
  C:1518H         LINE#         379
  C:151BH         LINE#         380
  C:151DH         LINE#         381
  C:1520H         LINE#         382
  -------         ENDPROC       TIMER1_1MS_POSLE_STARTOVANJA
  -------         PROC          EXTERN1_AUTOMAT_SPIRALA
  C:14ACH         LINE#         384
  C:14B0H         LINE#         385
  C:14B3H         LINE#         386
  C:14B6H         LINE#         387
  C:14B9H         LINE#         388
  C:14BCH         LINE#         389
  C:14BEH         LINE#         390
  C:14C0H         LINE#         391
  C:14C3H         LINE#         392
  C:14C5H         LINE#         393
BL51 BANKED LINKER/LOCATER V5.00                                                      02/17/2010  13:07:02  PAGE 11


  C:14C7H         LINE#         394
  C:14C7H         LINE#         395
  C:14CAH         LINE#         396
  -------         ENDPROC       EXTERN1_AUTOMAT_SPIRALA
  -------         PROC          _?EXTERN0_TASTATURA
  -------         DO            
  x:0000H         SYMBOL        temp_sec
  -------         ENDDO         
  C:0C79H         LINE#         398
  C:0C9CH         LINE#         399
  C:0C9FH         LINE#         400
  C:0CA2H         LINE#         401
  C:0CA5H         LINE#         403
  C:0CB9H         LINE#         405
  C:0CB9H         LINE#         406
  C:0CC5H         LINE#         407
  C:0CCDH         LINE#         408
  C:0CD5H         LINE#         409
  C:0CD7H         LINE#         410
  C:0CD7H         LINE#         411
  C:0CD7H         LINE#         412
  C:0CDAH         LINE#         414
  C:0CDAH         LINE#         415
  C:0CE3H         LINE#         416
  C:0D16H         LINE#         418
  C:0D20H         LINE#         419
  C:0D22H         LINE#         420
  C:0D24H         LINE#         421
  C:0D26H         LINE#         422
  C:0D4BH         LINE#         423
  C:0D4EH         LINE#         424
  C:0D7AH         LINE#         425
  C:0DACH         LINE#         426
  C:0DB4H         LINE#         427
  C:0DBBH         LINE#         428
  C:0DBBH         LINE#         429
  C:0DBDH         LINE#         430
  C:0DBDH         LINE#         431
  C:0DC4H         LINE#         432
  C:0DC4H         LINE#         433
  C:0DC4H         LINE#         434
  C:0DC6H         LINE#         435
  C:0DC6H         LINE#         436
  C:0DCFH         LINE#         437
  C:0DCFH         LINE#         438
  C:0DCFH         LINE#         439
  C:0DCFH         LINE#         440
  C:0DCFH         LINE#         441
  C:0DD1H         LINE#         443
  C:0DD1H         LINE#         444
  C:0DE1H         LINE#         445
  C:0DE4H         LINE#         446
  C:0DE7H         LINE#         447
  C:0DE7H         LINE#         448
  C:0DE9H         LINE#         449
  C:0DE9H         LINE#         450
  C:0DECH         LINE#         451
BL51 BANKED LINKER/LOCATER V5.00                                                      02/17/2010  13:07:02  PAGE 12


  C:0DEFH         LINE#         452
  C:0DF1H         LINE#         453
  C:0DFBH         LINE#         454
  C:0DFEH         LINE#         455
  C:0E01H         LINE#         456
  C:0E01H         LINE#         457
  C:0E01H         LINE#         458
  -------         ENDPROC       _?EXTERN0_TASTATURA
  -------         PROC          SERIJSKI_PORT
  -------         DO            
  D:0005H         SYMBOL        poruka
  -------         DO            
  X:0773H         SYMBOL        i
  X:0773H         SYMBOL        i
  X:0774H         SYMBOL        promet_u
  -------         ENDDO         
  -------         DO            
  X:0773H         SYMBOL        i
  X:0774H         SYMBOL        promet_u
  -------         ENDDO         
  -------         DO            
  X:0773H         SYMBOL        temp
  -------         ENDDO         
  -------         ENDDO         
  C:0A47H         LINE#         460
  C:0A5CH         LINE#         463
  C:0A62H         LINE#         464
  C:0A64H         LINE#         465
  C:0A6BH         LINE#         467
  C:0A6FH         LINE#         469
  C:0AA5H         LINE#         470
  C:0AA5H         LINE#         472
  C:0AAAH         LINE#         473
  C:0AAEH         LINE#         474
  C:0AB2H         LINE#         475
  C:0AF1H         LINE#         476
  C:0AF7H         LINE#         477
  C:0AFEH         LINE#         478
  C:0B01H         LINE#         479
  C:0B01H         LINE#         480
  C:0B03H         LINE#         481
  C:0B05H         LINE#         482
  C:0B08H         LINE#         483
  C:0B08H         LINE#         484
  C:0B2BH         LINE#         486
  C:0B2BH         LINE#         487
  C:0B30H         LINE#         488
  C:0B30H         LINE#         489
  C:0B30H         LINE#         490
  C:0B44H         LINE#         491
  C:0B71H         LINE#         492
  C:0B71H         LINE#         493
  C:0B78H         LINE#         494
  C:0B89H         LINE#         495
  C:0B89H         LINE#         496
  C:0B8CH         LINE#         497
  C:0B8CH         LINE#         498
BL51 BANKED LINKER/LOCATER V5.00                                                      02/17/2010  13:07:02  PAGE 13


  C:0B99H         LINE#         499
  C:0BAEH         LINE#         500
  C:0BAEH         LINE#         501
  C:0BAEH         LINE#         502
  C:0BAEH         LINE#         503
  C:0BB0H         LINE#         505
  C:0BB0H         LINE#         506
  C:0BB5H         LINE#         507
  C:0BB7H         LINE#         508
  C:0BB9H         LINE#         509
  C:0BBCH         LINE#         510
  C:0BCFH         LINE#         511
  C:0BD2H         LINE#         512
  C:0BD2H         LINE#         513
  C:0BD2H         LINE#         514
  C:0BD4H         LINE#         516
  C:0BD4H         LINE#         517
  C:0BDAH         LINE#         518
  C:0BDCH         LINE#         519
  C:0BEFH         LINE#         520
  C:0BF2H         LINE#         521
  C:0BF4H         LINE#         522
  C:0BF4H         LINE#         523
  C:0BF6H         LINE#         525
  C:0BF6H         LINE#         526
  C:0BFDH         LINE#         527
  C:0C02H         LINE#         528
  C:0C05H         LINE#         529
  C:0C05H         LINE#         530
  C:0C07H         LINE#         531
  C:0C0CH         LINE#         532
  C:0C11H         LINE#         533
  C:0C13H         LINE#         534
  C:0C15H         LINE#         535
  C:0C15H         LINE#         536
  C:0C1AH         LINE#         537
  C:0C1DH         LINE#         538
  C:0C1FH         LINE#         539
  C:0C22H         LINE#         540
  C:0C22H         LINE#         541
  C:0C24H         LINE#         543
  C:0C24H         LINE#         544
  C:0C41H         LINE#         545
  C:0C45H         LINE#         546
  C:0C48H         LINE#         547
  C:0C48H         LINE#         548
  C:0C48H         LINE#         549
  C:0C48H         LINE#         550
  C:0C4AH         LINE#         551
  C:0C4CH         LINE#         553
  C:0C4FH         LINE#         554
  C:0C51H         LINE#         555
  C:0C5BH         LINE#         557
  C:0C5BH         LINE#         558
  C:0C5BH         LINE#         559
  C:0C5BH         LINE#         560
  C:0C5BH         LINE#         561
BL51 BANKED LINKER/LOCATER V5.00                                                      02/17/2010  13:07:02  PAGE 14


  C:0C5DH         LINE#         562
  C:0C5DH         LINE#         563
  C:0C60H         LINE#         564
  C:0C63H         LINE#         565
  C:0C66H         LINE#         566
  C:0C66H         LINE#         567
  C:0C66H         LINE#         568
  C:0C66H         LINE#         569
  -------         ENDPROC       SERIJSKI_PORT
  -------         ENDMOD        AUTOMAT

  -------         MODULE        ?C?COPY
  C:08D0H         PUBLIC        ?C?COPY
  -------         ENDMOD        ?C?COPY

  -------         MODULE        ?C?SCDIV
  C:08F6H         PUBLIC        ?C?SCDIV
  -------         ENDMOD        ?C?SCDIV

  -------         MODULE        ?C?CLDOPTR
  C:0918H         PUBLIC        ?C?CLDOPTR
  -------         ENDMOD        ?C?CLDOPTR

  -------         MODULE        ?C?IMUL
  C:0945H         PUBLIC        ?C?IMUL
  -------         ENDMOD        ?C?IMUL

  -------         MODULE        ?C?SIDIV
  C:0957H         PUBLIC        ?C?SIDIV
  -------         ENDMOD        ?C?SIDIV

  -------         MODULE        ?C?IILDX
  C:098DH         PUBLIC        ?C?IILDX
  -------         ENDMOD        ?C?IILDX

  -------         MODULE        ?C_XBP
  D:0017H         PUBLIC        ?C_XBP
  -------         ENDMOD        ?C_XBP

  -------         MODULE        ?C?ADDXBP
  C:09A3H         PUBLIC        ?C?ADDXBP
  -------         ENDMOD        ?C?ADDXBP

  -------         MODULE        STRCAT
  D:0008H         PUBLIC        ?_strcat?BYTE
  C:13F5H         PUBLIC        _strcat
  -------         ENDMOD        STRCAT

  -------         MODULE        ?C?CLDPTR
  C:09C7H         PUBLIC        ?C?CLDPTR
  -------         ENDMOD        ?C?CLDPTR

  -------         MODULE        ?C?CSTPTR
  C:09E0H         PUBLIC        ?C?CSTPTR
  -------         ENDMOD        ?C?CSTPTR

  -------         MODULE        ?C?UIDIV
BL51 BANKED LINKER/LOCATER V5.00                                                      02/17/2010  13:07:02  PAGE 15


  C:09F2H         PUBLIC        ?C?UIDIV
  -------         ENDMOD        ?C?UIDIV

******************************************************************************
* RESTRICTED VERSION WITH 0800H BYTE CODE SIZE LIMIT; USED: 0A33H BYTE (127%) *
******************************************************************************

Program Size: data=76.3 xdata=1910 code=3388
LINK/LOCATE RUN COMPLETE.  0 WARNING(S),  0 ERROR(S)

*** FATAL ERROR L250: CODE SIZE LIMIT IN RESTRICTED VERSION EXCEEDED
    MODULE:  C:\KEIL\C51\LIB\C51S.LIB (-----)
    LIMIT:   0800H BYTES